:1000000012C01895189518951895189547C0189509
:100010001895189518951895189518951895189578
:100020001895189518958FED8DBFC0ECE0EC4E2E0D
:10003000DD275D2EEEE7F0E0A0E6B0E088278D93A7
:100040003197E9F783E389B980E082B988E18AB919
:1000500066248FEF87BB8FEF88BB8FEB81BB8FEF61
:1000600082BB789449D0A0E62C93A1E61C93A1E62C
:100070008C918F778C9300916000003009F00BC059
:10008000C79831E0A1E617D082E390E026D0C79A66
:1000900082E390E022D0E6CFF894FFCF8F939F9336
:1000A0008FB73395539509F4439591E892BF9F918B
:1000B0008FBF8F9118958D9103D03A95E1F70895F0
:1000C0005D9BFECF8CB908953197F1F70895689440
:1000D00062F80895E89462F80895EF93FF93EE278D
:1000E000E82BE92B31F0E0EAFFE03197F1F70197D7
:1000F000D1F7FF91EF9108950F933F934F935F9343
:100100002F923F928F939F938FB78F9383B78F9345
:10011000826083BF89B78F93826089BF81E882BF85
:10012000552744273327483008F047C0373324F495
:10013000869BF8CFF8CF41C04830ECF78699FCCFCA
:1001400033273232D4F5869BFCCF932F33271127E8
:100150002227913110F0969511E0292E2694322C09
:10016000290E990F390E113021F0321534F5869988
:10017000FCCF33270CE03215F0F3869909C0889440
:10018000111F221F3315CCF4869BFCCF332708C0E8
:100190000894111F221F331584F48699FCCF33274E
:1001A0000A9549F7912F991F221F991F221F25FB9E
:1001B00017F926FB16F92F7102C01FEF2FEF8F9151
:1001C00089BF8F9183BF8F918FBF9F918F913F90F8
:0C01D0002F905F914F913F910F91089587
:00000001FF
